:10E000008E00FFBDE74CCE0000DFD0DFD7DFD58626
:10E010005397D97F00DB7F00DC7F00DDDFDE9FE0F0
:10E02000DFE286C097E4CEE663BDE54CCE55AAC6D6
:10E030006486058B05188155271F816E2714811072
:10E040002625CEFFFFEC018C00002714CEE6CF4F33
:10E05000201CCEE6D886012015CEE6E18603200EF0
:10E06000CEE6EA86042007BDE55ACEE6C54F97DB2B
:10E07000BDE54CCEE67EBDE54CBDE59FCE00C0BD06
:10E08000E5E6BDE5F04D27EB814426037EE0BA814D
:10E090004726037EE1D6815326037EE209814C2682
:10E0A000037EE271815026037EE362815226037E65
:10E0B000E473CEE69BBDE54C20B908BDE5E6BDE5C1
:10E0C000FB5D2615BDE5E6A60026E796D18B809779
:10E0D000D396D0890097D2203896E697D196E597C7
:10E0E000D0BDE5E6A600812C27114D26C596D18B23
:10E0F0008097D396D0890097D2201608BDE5E6BD5B
:10E10000E5FBBDE5E65D27AA6D0026A6DEE508DF96
:10E11000D296D184F097E896D097E77F00D48D21EE
:10E12000BDE75E261196D4810225F396D397D1964A
:10E13000D297D07EE07396E897D196E797D07EE0AD
:10E140007396E7D6E8BDE557CEE6A3BDE54CCE0015
:10E15000C0DFE9C6108D295A26FBCEE6A6BDE54CE8
:10E16000CE00C0C610A6000881202509817F2405A5
:10E17000BDE7632005862EBDE7635A26E87EE59558
:10E180008620BDE76396D4262596D091E72606968D
:10E19000D191E827158620BDE763BDE763DEE9A7D7
:10E1A0000008DFE9DEE708DFE739860197D496D477
:10E1B000810126E1DEE7A60008DFE7DEE9A7000827
:10E1C000DFE9BDE55A96D291E7260A96D391E82673
:10E1D00004860297D43908BDE5E6BDE5FBA6002715
:10E1E000037EE0B25D2704DEE5DFE296E09AE127F8
:10E1F000029EE096E33696E23696DF3696DE369657
:10E20000DC3696DD3696E4363B08BDE5E6BDE5FB3B
:10E21000BDE5E66D0026575D2704DEE5DFD796D71E
:10E22000D6D8BDE557CEE6A6BDE54CDED7A600BDE7
:10E23000E55A8620BDE763BDE59FCE00C0BDE5E69B
:10E24000A6002607DED708DFD720D3812D2607DEDC
:10E25000D709DFD720C8812E26037EE073BDE5FBFA
:10E260005D270BDED796E6A70008DFD720B07EE05B
:10E27000B208BDE5E6BDE5FBBDE5E66D0026EFBDF8
:10E28000E755BDE5F08153276F813A270D810D27B2
:10E29000EE810A27EABDE75520F3BDE56F97EB163F
:10E2A000BDE56F97E79BEB97EBBDE56F97E89BEBC1
:10E2B00097EB96E89BE697E896E799E597E7DEE720
:10E2C000BDE56F97DA9BEB97EB5D2714BDE56F36E5
:10E2D0009BEB97EB327D00DA2603A700085A26EC69
:10E2E000BDE56F9BEB26087D00DA27A97EE073CEA3
:10E2F000E681BDE54C7EE073BDE75597DABDE56F7D
:10E300001697EBBDE56F97E79BEB97EBBDE56F9736
:10E31000E89BEB97EB96E89BE697E896E799E597FD
:10E32000E7DEE7C0032718BDE56F369BEB97EB965A
:10E33000DA8131260632A700082001325A26E8BDCC
:10E34000E56F9BEB81FF261196DA81372711813823
:10E35000270D813927097EE295CEE68EBDE54C7EFC
:10E36000E07308A600BDE5F0814927048153260328
:10E370000897D9BDE5E6BDE5FB5D272296E597E95F
:10E3800096E697EABDE5E6A600812C261108BDE5D4
:10E39000E6BDE5FB5D2707BDE5E66D0027037EE0F2
:10E3A000B2DEE508DFE596E690EA97E696E592E9C3
:10E3B00097E5DEE98D1E96E59AE626F896D981491D
:10E3C0002609CEE6AABDE54C7EE073CEE6B8BDE5F3
:10E3D0004C7EE073C6107D00E5260696E61124010A
:10E3E0001696E61097E696E5820097E596D981495C
:10E3F000263F863ABDE76317BDE55AD7EBDFE996BE
:10E40000E9BDE55A96E99BEB97EB96EABDE55A968E
:10E41000EA9BEB97EB4FBDE55AA60036BDE55A32B5
:10E420009BEB97EB085A26F196EB40BDE55A7EE54B
:10E43000958653BDE7638631BDE763178B0397EB82
:10E44000BDE55ADFE996E9BDE55A96E99BEB97EB06
:10E4500096EABDE55A96EA9BEB97EBA60036BDE53A
:10E460005A329BEB97EB085A26F196EB43BDE55ADF
:10E470007EE59508BDE5E6BDE5F04D2606BDE50166
:10E480007EE073DFE7CEE7146D002772A100270856
:10E4900008080808080820F0DFE9DEE708BDE5E61F
:10E4A0006D00265ADEE9EE04BDE54C863DBDE7630E
:10E4B000DEE9E601EE02C1012607A600BDE55A200D
:10E4C0000AA600BDE55AA601BDE55A8620BDE76350
:10E4D000BDE59FCE00C0BDE5E6A600271EBDE5FB5D
:10E4E0005D271BDEE9E601EE02C101260696E6A7DE
:10E4F00000200896E5A70096E6A7017EE0737EE07F
:10E50000B2CEE6F9BDE54C96DCBDE55ACEE6FCBDE3
:10E51000E54C96DDBDE55ACEE700BDE54C96DED66E
:10E52000DFBDE557CEE704BDE54C96E0D6E1BDE59D
:10E5300057CEE709BDE54C96E2D6E3BDE557CEE7F9
:10E540000EBDE54C96E4BDE55A7EE595A60027068E
:10E55000BDE7630820F6398D011736444444448DE5
:10E560000132840F8B30813A25028B077EE7634F9F
:10E570008D04484848483716BDE755BDE5F0813061
:10E580002511813A250A8141250981472405800703
:10E5900080301B3339860DBDE763860A7EE763CE84
:10E5A00000C05FBDE755810D2737810A27338108F9
:10E5B0002719817F2715812025E9818024E5C10F56
:10E5C00024E15CA70008BDE76320D85D27D55A0980
:10E5D0008608BDE7638620BDE7638608BDE7632044
:10E5E000C28DB26F0039A600812026030820F739BA
:10E5F00081612506817B24028BE0395F7F00E57F06
:10E6000000E6A6008DEA81302534813A250A814151
:10E61000252C814724288007803049494949497978
:10E6200000E67900E5497900E67900E5497900E6F8
:10E630007900E5497900E67900E5085C20C439CE27
:10E64000E6F3BDE54C3297E43297DD3297DC329742
:10E65000DE3297DF3297E23297E39FE0BDE5017E3D
:10E66000E0733B0D0A556E6976657273616C204DDF
:10E670006F6E69746F7220363830300D0A005D207D
:10E68000004572726F7220696865780D0A004572E4
:10E69000726F7220737265630D0A004572726F7239
:10E6A0000D0A00203A00203A20003A303030303055
:10E6B00030303146460D0A00533930333030303077
:10E6C00046430D0A00556E6B6E6F776E0D0A004D56
:10E6D00043363830300D0A004D43363830310D0A9C
:10E6E000004844363330310D0A004D423838363157
:10E6F0000D0A005357490D0A00413D0020423D00DC
:10E7000020583D002053503D002050433D00204301
:10E7100043523D00410100DCE73C420100DDE73EA1
:10E72000580200DEE740530200E0E742500200E0FA
:10E73000E745430100E4E7480000000041004200D3
:10E740005800535000504300434352008605971031
:10E75000860A9711399611848027FA9612399611F4
:0EE76000848039369611842027FA32971339B7
:03FF80007EE00020
:03FF88007EE073A5
:03FF90007EE763A6
:03FF98007EE54CB7
:03FFA0007EE755A4
:03FFA8007EE75E93
:08FFF800E662E63FE662E0006C
:00000001FF
